:100000001FC012C411C410C40FC40EC40DC40CC44C
:100010000BC40AC409C408C407C406C405C404C484
:1000200003C402C401C400C4FFC3FEC3FDC3FCC3B8
:10003000FBC3FAC33F003F10803F103F140008325B
:1000400011241FBECFEFCDBFDFE3DEBFE4E3F0E05E
:1000500040E017C0B591A59135912591059107FD17
:100060000CC095918591EF01F92FE82F05900D9225
:10007000A217B307D9F7FE0104C01D92A217B30758
:10008000E1F7E034F40731F709D28EC3F894FFCFDB
:100090004F925F926F927F928F929F92AF92BF9298
:1000A000CF92DF92EF92FF92CF936B017C0123EE10
:1000B00038E34EE85FE3B6D34B015C0120E030E06B
:1000C00040E85FE39CD388230CF464C024E535E565
:1000D00045E55FE3C701B601A5D32B013C0120E054
:1000E0003FEF4FE757E48FD318160CF03EC020E0E7
:1000F00030E04AE754E4C701B60192D34B015C01FA
:1001000024E535E540E554E48DD36B017C0120E026
:1001100030E040E85FE373D388230CF120E03FEF49
:100120004FE757E4C701B6016ED31816A4F420E0D8
:1001300030E040E251E4C501B40174D3DCD1611573
:10014000710549F123E530E0C9010197F1F76150EC
:100150007109D1F720C0C701B601CDD102C061E05D
:1001600070E0CB010197F1F716C020E030E04FE7D7
:1001700053E4C501B40147D318163CF4C301B201DE
:10018000BAD1CB010197F1F709C0C501B401B3D1D0
:10019000C62F01C0C1E06C2F6A95F1F7CF91FF9097
:1001A000EF90DF90CF90BF90AF909F908F907F9017
:0801B0006F905F904F900895DD
:1001B8000BC0E8D240F0DFD230F021F45F3F19F0F5
:1001C800FCC25111E7C225C308D298F39923C9F399
:1001D8005523B1F3951B550BBB27AA276217730745
:1001E800840738F09F5F5F4F220F331F441FAA1FF9
:1001F800A9F333D00E2E3AF0E0E830D091505040B9
:10020800E695001CCAF729D0FE2F27D0660F771F66
:10021800881FBB1F261737074807AB07B0E809F048
:10022800BB0B802DBF01FF2793585F4F2AF09E3FDD
:10023800510568F0C2C2AEC25F3FECF3983EDCF3F2
:10024800869577956795B795F7959F5FC9F7880F56
:10025800911D9695879597F90895E1E0660F771FA8
:10026800881FBB1F621773078407BA0720F0621B39
:0E027800730B840BBA0BEE1F88F7E095089508
:100286000AC07AD228F07FD218F0952309F096C2D8
:10029600C1C2112480C2A2D1A0F3959FD1F3950FBC
:1002A60050E0551F629FF001729FBB27F00DB11DF4
:1002B600639FAA27F00DB11DAA1F649F6627B00D84
:1002C600A11D661F829F2227B00DA11D621F739F6D
:1002D600B00DA11D621F839FA00D611D221F749F7B
:1002E6003327A00D611D231F849F600D211D822FC2
:1002F600762F6A2F11249F5750408AF0E1F0882309
:100306004AF0EE0FFF1FBB1F661F771F881F915015
:100316005040A9F79E3F510570F050C23CC25F3F66
:10032600ECF3983EDCF3869577956795B795F79548
:10033600E7959F5FC1F7FE2B880F911D96958795D0
:0403460097F9089586
:10034A00E89409C097FB3EF4909580957095619565
:10035A007F4F8F4F9F4F9923A9F0F92F96E9BB271B
:10036A009395F695879577956795B795F111F8CF97
:10037A00FAF4BB0F11F460FF1BC06F5F7F4F8F4F02
:10038A009F4F16C0882311F096E911C0772321F0F8
:10039A009EE8872F762F05C0662371F096E8862F90
:1003AA0070E060E02AF09A95660F771F881FDAF7E7
:0A03BA00880F9695879597F908952E
:1003C4000F931F93CF93DF93C82FD62F71D102D2EF
:1003D4008C2F93D1E091123FF091133F8C2F09950C
:1003E4008C01FDD100511240083D114080F4EC2FE6
:1003F400F0E0E85FF04C8081811109C06D2F80E04E
:1004040094E0AFD16D2F84E094E0ABD10AC06D2F9E
:1004140084E094E07FD1EC2FF0E0E85FF04C81E0E1
:0C0424008083DF91CF911F910F9108950C
:100430000F931F93CF93DF93C82FD62F3BD1CCD1EF
:100440008C2F5DD1E091123FF091133F8C2F0995D5
:100450008C01C7D100511240083D114080F4EC2FAF
:10046000F0E0E050F14C8081811109C06D2F80E2F5
:1004700094E079D16D2F84E294E075D10AC06D2F9C
:1004800084E294E049D1EC2FF0E0E050F14C81E0BF
:0C0490008083DF91CF911F910F910895A0
:10049C004AD1C3D0CEECD7E808ED17E80F2EFAED11
:1004AC00EF2EFAE1FF2EF02DA0D1C7010197F1F745
:1004BC003AD146D189919991E1D0C017D107A1F7D2
:1004CC0088EA91E623E530E0F9013197F1F70197DD
:1004DC00D9F78BD128D161E084E06EDF63E085E051
:0A04EC00A1DF62E086E09EDFF6CF9C
:1004F6007DD088F09F5790F0B92F9927B751A0F07B
:10050600D1F0660F771F881F991F1AF0BA95C9F7A1
:1005160012C0B13081F03ED1B1E008953BC1672FE2
:10052600782F8827B85F39F0B93FCCF38695779551
:100536006795B395D9F73EF490958095709561953A
:080546007F4F8F4F9F4F089576
:10054E000F931F93CF93DF932FD1E091123FF09132
:10055E00133F87E009958C013DD126D1E091123FE2
:10056E00F091133F87E00995EC0134D1C11582E07B
:10057E00D80730F081E0C017D10718F480E001C031
:0C058E0080E0DF91CF911F910F91089544
:10059A00990F0008550FAA0BE0E8FEEF161617068A
:1005AA00E807F907C0F012161306E407F50798F0F2
:1005BA00621B730B840B950B39F40A2661F0232B0B
:1005CA00242B252B21F408950A2609F4A140A69587
:0805DA008FEF811D811D0895C2
:1005E20057FD9058440F551F59F05F3F71F04795E2
:1005F200880F97FB991F61F09F3F79F087950895C7
:10060200121613061406551FF2CF4695F1DF08C0E5
:10061200161617061806991FF1CF86957105610502
:04062200089408959B
:1006260060E080E096E0F3D065E081E096E0EFD010
:1006360064E082E096E094D062E082E096E090D0BA
:1006460060E483E096E0CFD064E083E096E088D073
:02065600089505
:1006580061E088E096E0DAD0E0E0F6E0838580FFAC
:10066800FDCFE0E0F6E081E0838780899189969567
:100678008795929582958F7089279F70892708950D
:10068800BC0180E090E05DDEE091103FF091113F09
:10069800099561E084E094E03BD063E084E294E073
:0C06A80037D062E084E294E033D0089583
:1006B400CF93883078F4C82F682F80E094E02AD054
:1006C4006C2F84E094E026D08C2F90E064E0805F6F
:0806D4009B4F47D0CF91089520
:1006DC00092E0394000C11F4882352F0BB0F40F444
:1006EC00BF2B11F460FF04C06F5F7F4F8F4F9F4F84
:0206FC0008955F
:1006FE00CF93883040F4C82F86E096E081D06C2FDF
:0A070E0086E096E080D0CF910895B8
:1007180021E030E002C0220F331F6A95E2F72095EE
:0A072800FC01308123232083089593
:1007320061E080E094E016D063E080E294E012D0C1
:0A07420062E080E294E00ED008951A
:10074C0061E084E094E009D063E084E294E005D0B9
:0A075C0062E084E294E001D0089509
:1007660021E030E002C0220F331F6A95E2F7FC0158
:080776003081232B208308953C
:0E077E0000240A941616170618060906089598
:0E078C0000240A94121613061406050608959A
:0E079A00E894BB2766277727CB0197F90895CF
:0E07A800EC0140D03ED0CE013ED0CE013DD07F
:0C07B60087E07DDF87E0A0DF0CD0089515
:0C07C20097F99F6780E870E060E0089500
:0A07CE00FA00F401EE02E803E20471
:0A07D80060E080E096E0C3DF0895C2
:0A07E20060E080E096E097DF0895E4
:0A07EC00FC012081622B6083089558
:0807F600ABDE8823E9F308954E
:0807FE00CDDE08F481E008954E
:08080600C9DE08F48FEF08952C
:06080E00FC0110820895B8
:06081400FC016083089561
:06081A009FEF80EC089541
:04082000CBDC5CCF02
:0408240030DD5ACF9A
:02082800EBCB18
:02082A0008952F
:02082C0008952D
:02082E0008952B
:020830002DDCBD
:0208320048007C
:020834002C0393
:00000001FF
